:020000003528A1
:10000800080003178C0083168C130C1555308D00CF
:10001800AA308D008C148C180F280C113028A301DD
:10002800A200FF30A207031CA307031C30280330DB
:10003800A100E73021201528A101FC3EA000A1095C
:10004800031C2C28FF300000A00703182728A0074E
:100058006400A10F26280800831303138312640089
:100068000800831607309F009901831298018316B0
:10007800023098008312BD01BC01BE0164008130CA
:100088003E028A110A120318EB283E08803C8A11A6
:100098000A12031CDB288A110A125620BD008A1195
:1000A8000A12DB2800308A003E0882071F34113408
:1000B8001F3401341F3400341D34153417341534FB
:1000C80015341F340C340A341F34173415341D34D6
:1000D8001F3415341C341934053403341F341534D3
:1000E8001F34173415341F340034003400340034FE
:1000F8000034003400340034003400340034003458
:100108000034003400340034003400340034003447
:1001180000341E3405341E341F3415340E341F3495
:10012800113411341F3411340E341F341534113482
:100138001F34053401341F3411341D341F34043482
:100148001F3411341F341134183410341F341F3441
:100158000A3411341F34103410341F3406341F3459
:100168001F340E341F340E3411340E341F3405344A
:1001780002340E34093416341F3405341B34163453
:1001880015340D3401341F3401341F3410341F3436
:100198000F3410340F341F3408341F341B34043424
:1001A8001B3403341C3403341934153413343C0819
:1001B80003178D0003133D088A0105200A308A01C0
:1001C8001320BC0ABE0A8A110A12031D42286300C2
:0401D8008A01EB2885
:02400E00753DFE
:00000001FF
